:100000007F28FF3E031D012808000739820780343E
:1000100001344034023420340434103408340F39AD
:1000200082073F3406345B344F3466346D347D349C
:1000300007347F34003401344034083438347934A0
:10004000733403141408FF39031D08000800083036
:1000500091001103203E84000008073911020800B6
:100060000800FF30900017080F2005118600851446
:10007000FF300120170E0F20851086000515FF3078
:100080000120900B332808000A3091004C28910B76
:100090004C28160894040B343030900006081605DE
:1000A000031D5728900B4E28160894040C34C030BA
:1000B00090000608160503194728900B59285D3053
:1000C00090001608060503196A28900B6228160886
:1000D00094040A340730910090010630012000009A
:1000E00000000000031016080605031D0314900D00
:1000F00003300120910B6F28100A0F390800950179
:1001000094018316811301308500FF30860083122D
:100110008501150805209600442097001508203E0B
:10012000840017088000950A15080739031D8928DF
:1001300083168601831205309100A628283091008D
:10014000513097003120910BA028B928950115084E
:10015000203E840000080F399700150E103EF0393C
:1001600097043120950A1508083A031DA728910B1A
:10017000A6289530970031205D3097003120DE3081
:1001800097003120EE3097003120EF30970031207A
:0C0190008316FF30850086008312630098
:02400E00F23F7F
:00000001FF
